:100000002500D70C0200A304E90C0600000C260012
:1000100067000607080A0000E703090A69000606E8
:100020000F0A110C2700E702130A0606030A080C40
:100030002800200C2700E7021B0A2A03EA0406070F
:10004000EA05E802190A220C2700E702250A000047
:100050000607030AA902C900070EE201360A370A99
:10006000380A390A3A0A4B0A4C0A4D0A0F0A0F0A93
:100070000F0A0F0A040C8A004307410A26054604AA
:100080004A0A140C8A004307480A260446054A0A0D
:0E009000260446040F0A0F0A0F0A6900080A28
:021FFE00EA0FE8
:00000001FF
